BL51 BANKED LINKER/LOCATER V6.22                                                        12/08/2025  20:07:38  PAGE 1


BL51 BANKED LINKER/LOCATER V6.22, INVOKED BY:
C:\KEIL\C51\BIN\BL51.EXE te.obj TO pro RAMSIZE (256)


MEMORY MODEL: SMALL


INPUT MODULES INCLUDED:
  te.obj (TE)
  C:\KEIL\C51\LIB\C51S.LIB (?C_STARTUP)


LINK MAP OF MODULE:  pro (TE)


            TYPE    BASE      LENGTH    RELOCATION   SEGMENT NAME
            -----------------------------------------------------

            * * * * * * *   D A T A   M E M O R Y   * * * * * * *
            REG     0000H     0008H     ABSOLUTE     "REG BANK 0"
                    0008H     0028H                  *** GAP ***
            DATA    0030H     0001H     ABSOLUTE     
                    0031H     006BH                  *** GAP ***
            IDATA   009CH     0001H     ABSOLUTE     
            IDATA   009DH     0001H     UNIT         ?STACK

            * * * * * * *  X D A T A   M E M O R Y  * * * * * * *
                    0000H     1130H                  *** GAP ***
            XDATA   1130H     0001H     ABSOLUTE     

            * * * * * * *   C O D E   M E M O R Y   * * * * * * *
            CODE    0000H     0003H     ABSOLUTE     
            CODE    0003H     000CH     UNIT         ?C_C51STARTUP
            CODE    000FH     000AH     UNIT         ?PR?RAM_LOW128BDATA?TE
            CODE    0019H     0009H     UNIT         ?PR?MAIN?TE
            CODE    0022H     0009H     UNIT         ?PR?RAM_HI128BDATA?TE
            CODE    002BH     0009H     UNIT         ?PR?XRAM_FUN?TE



OVERLAY MAP OF MODULE:   pro (TE)


SEGMENT
  +--> CALLED SEGMENT
---------------------
?C_C51STARTUP
  +--> ?PR?MAIN?TE

?PR?MAIN?TE
  +--> ?PR?RAM_LOW128BDATA?TE
  +--> ?PR?RAM_HI128BDATA?TE
  +--> ?PR?XRAM_FUN?TE



SYMBOL TABLE OF MODULE:  pro (TE)

BL51 BANKED LINKER/LOCATER V6.22                                                      12/08/2025  20:07:38  PAGE 2


  VALUE           TYPE          NAME
  ----------------------------------

  -------         MODULE        TE
  C:0000H         SYMBOL        _ICE_DUMMY_
  D:0080H         PUBLIC        P0
  D:0090H         PUBLIC        P1
  D:00A0H         PUBLIC        P2
  D:00B0H         PUBLIC        P3
  D:00C0H         PUBLIC        P4
  D:00C8H         PUBLIC        P5
  D:00E8H         PUBLIC        P6
  D:00F8H         PUBLIC        P7
  D:00A8H         PUBLIC        IE
  C:0022H         PUBLIC        RAM_hi128Bdata
  C:000FH         PUBLIC        RAM_low128Bdata
  D:00B8H         PUBLIC        IP
  D:00D8H         PUBLIC        CCON
  C:0019H         PUBLIC        main
  I:009CH         PUBLIC        x1
  D:0030H         PUBLIC        x2
  X:1130H         PUBLIC        x3
  D:0098H         PUBLIC        SCON
  D:0088H         PUBLIC        TCON
  C:002BH         PUBLIC        XRAM_fun
  D:00D0H         PUBLIC        PSW
  -------         PROC          MAIN
  C:0019H         LINE#         10
  C:0019H         LINE#         13
  C:001CH         LINE#         15
  C:001FH         LINE#         17
  -------         ENDPROC       MAIN
  -------         PROC          RAM_LOW128BDATA
  -------         DO            
  D:0000H         SYMBOL        p
  -------         ENDDO         
  C:000FH         LINE#         26
  C:000FH         LINE#         30
  C:0011H         LINE#         31
  C:0013H         LINE#         35
  C:0015H         LINE#         38
  C:0018H         LINE#         40
  -------         ENDPROC       RAM_LOW128BDATA
  -------         PROC          RAM_HI128BDATA
  -------         DO            
  D:0000H         SYMBOL        p
  -------         ENDDO         
  C:0022H         LINE#         43
  C:0022H         LINE#         48
  C:0024H         LINE#         49
  C:0026H         LINE#         60
  C:002AH         LINE#         63
  -------         ENDPROC       RAM_HI128BDATA
  -------         PROC          XRAM_FUN
  -------         DO            
  D:0082H         SYMBOL        p
  -------         ENDDO         
BL51 BANKED LINKER/LOCATER V6.22                                                      12/08/2025  20:07:38  PAGE 3


  C:002BH         LINE#         66
  C:002BH         LINE#         71
  C:002EH         LINE#         72
  C:0031H         LINE#         82
  C:0032H         LINE#         85
  C:0033H         LINE#         87
  -------         ENDPROC       XRAM_FUN
  -------         ENDMOD        TE

Program Size: data=11.0 xdata=1 code=52
LINK/LOCATE RUN COMPLETE.  0 WARNING(S),  0 ERROR(S)
